
 Start         Length     Name                   Class
 0003:00000000 000032C1H  _TEXT                  CODE 32-bit
 0003:000032C4 00000258H  ICODE                  ICODE 32-bit
 0004:00000000 00000004H  .CRT$XIA               DATA 32-bit
 0004:00000010 00000004H  .CRT$XIZ               DATA 32-bit
 0004:00000020 00000004H  .CRT$XCA               DATA 32-bit
 0004:00000030 00000004H  .CRT$XCZ               DATA 32-bit
 0004:00000040 00000004H  .CRT$XPA               DATA 32-bit
 0004:00000050 00000004H  .CRT$XPZ               DATA 32-bit
 0004:00000060 00000004H  .CRT$XTA               DATA 32-bit
 0004:00000070 00000004H  .CRT$XTZ               DATA 32-bit
 0004:00000074 00000000H  IMP__DATA              IMP__DATA 32-bit
 0004:00000080 00001654H  _DATA                  DATA 32-bit
 0004:000016E0 00000000H  FHB                    DATA 32-bit
 0004:000016E0 0000000CH  FH                     DATA 32-bit
 0004:000016EC 00000000H  FHE                    DATA 32-bit
 0004:000016F0 00000000H  FJB                    DATA 32-bit
 0004:000016F0 00000004H  FJ                     DATA 32-bit
 0004:000016F4 00000004H  FJE                    DATA 32-bit
 0004:000016F8 00000000H  XIFCB                  DATA 32-bit
 0004:000016F8 00000004H  XIFU                   DATA 32-bit
 0004:000016FC 00000000H  XIFL                   DATA 32-bit
 0004:000016FC 00000000H  XIFM                   DATA 32-bit
 0004:000016FC 00000000H  XIFCE                  DATA 32-bit
 0004:000016FC 00000000H  XIB                    DATA 32-bit
 0004:000016FC 00000000H  XI                     DATA 32-bit
 0004:000016FC 00000000H  XIE                    DATA 32-bit
 0004:000016FC 00000000H  XCB                    DATA 32-bit
 0004:000016FC 00000004H  XC                     DATA 32-bit
 0004:00001700 00000000H  XCE                    DATA 32-bit
 0004:00001700 00000000H  CONST                  CONST 32-bit
 0004:00001700 00000000H  EEND                   ENDBSS 32-bit
 0004:00001700 000006B0H  _BSS                   BSS 32-bit
 0004:00001DB0 00000000H  XOB                    BSS 32-bit
 0004:00001DB0 00000004H  XO                     BSS 32-bit
 0004:00001DB4 00000000H  XOE                    BSS 32-bit
 0004:00001DB4 00000000H  XOFB                   BSS 32-bit
 0004:00001DB4 00000104H  XOF                    BSS 32-bit
 0004:00001EB8 00000000H  XOFE                   BSS 32-bit
 0004:00001EC0 000007A9H  c_common               BSS 32-bit
 0004:00002670 00000000H  STACK                  STACK 32-bit

 Address       Export                  Alias

 0004:00000D30 $ClassNwQuotaD          _$ClassNwQuotaD
 0004:000016E0 $NwQuotaD_VERSION_1NUMBER  _$NwQuotaD_VERSION_1NUMBER
 0003:00000018 $NwQuotaD__4clinit_5__  _$NwQuotaD__4clinit_5__
 0003:0000004C $NwQuotaD__4init_5__    _$NwQuotaD__4init_5__
 0003:000004C0 $NwQuotaD_dumpToFile__Ljava_lang_String_2  _$NwQuotaD_dumpToFile__Ljava_lang_String_2
 0004:000016E4 $NwQuotaD_filter        _$NwQuotaD_filter
 0004:00000085 $NwQuotaD_filtrePositif  _$NwQuotaD_filtrePositif
 0003:000005C4 $NwQuotaD_getCurrentDateFormated__  _$NwQuotaD_getCurrentDateFormated__
 0004:000016E8 $NwQuotaD_logFileName   _$NwQuotaD_logFileName
 0003:0000060C $NwQuotaD_main___3Ljava_lang_String_2  _$NwQuotaD_main___3Ljava_lang_String_2
 0003:00000848 $NwQuotaD_parseArgs___3Ljava_lang_String_2  _$NwQuotaD_parseArgs___3Ljava_lang_String_2
 0004:00000080 $NwQuotaD_port          _$NwQuotaD_port
 0004:00000084 $NwQuotaD_showOnlyAlert  _$NwQuotaD_showOnlyAlert
 0004:00000F80 _vtbl_$ClassNwQuotaD    __vtbl_$ClassNwQuotaD

  Address         Publics by Name               Rva+Base

 0003:00002D90       ??0RTLHeap@@QAE@XZ         00405D90
 0003:00003010       ??0RTLHeapBlock@@QAE@IAAV0@@Z 00406010
 0003:00002FFC       ??0RTLHeapBlock@@QAE@XZ    00405FFC
 0003:00002FE0       ??0RTLHeapBlockHeader@@QAE@I@Z 00405FE0
 0003:00002568       ??0RTLMultiPool@@QAE@II@Z  00405568
 0003:00002C5C       ??0RTLPool@@QAE@II@Z       00405C5C
 0003:000025EC       ??1RTLMultiPool@@QAE@XZ    004055EC
 0003:00002DE8       ?Alloc@RTLHeap@@QAEPAXK@Z  00405DE8
 0003:000025F0       ?Alloc@RTLMultiPool@@QAEPAXK@Z 004055F0
 0003:00002D4C       ?Alloc@RTLPool@@QAEPAXXZ   00405D4C
 0003:00003108       ?Claim@RTLHeapBlock@@QAEHI@Z 00406108
 0003:000031B0       ?CreateMainHeap@RTLHeap@@SAXXZ 004061B0
 0003:000027B4       ?CreateMainHeap@RTLMultiPool@@SAXXZ 004057B4
 0003:00002DAC       ?FixSize@RTLHeap@@AAEII@Z  00405DAC
 0003:00002F90       ?Free@RTLHeap@@QAEXPAX@Z   00405F90
 0003:0000279C       ?Free@RTLMultiPool@@QAEXPAX@Z 0040579C
 0003:00002D7C       ?Free@RTLPool@@QAEXPAX@Z   00405D7C
 0003:000030E4       ?GetNext@RTLHeapBlock@@QAEAAV1@XZ 004060E4
 0003:00003030       ?InsertAfter@RTLHeapBlock@@QAEXAAV1@@Z 00406030
 0003:00003058       ?MergeBackward@RTLHeapBlock@@QAEHXZ 00406058
 0003:00003098       ?MergeForward@RTLHeapBlock@@QAEHXZ 00406098
 0003:00002F20       ?MoreCore@RTLHeap@@AAEPAVRTLHeapBlock@@I@Z 00405F20
 0003:00002E4C       ?Realloc@RTLHeap@@QAEPAXPAXK@Z 00405E4C
 0003:00002640       ?Realloc@RTLMultiPool@@QAEPAXPAXK@Z 00405640
 0003:0000313C       ?Reclaim@RTLHeapBlock@@QAEHIAAV1@@Z 0040613C
 0003:000030EC       ?Remove@RTLHeapBlock@@QAEXXZ 004060EC
 0003:00002760       ?SelectFree@RTLMultiPool@@AAEXPAX@Z 00405760
 0003:00002CC0       ?ThreadNewBlock@RTLPool@@AAEXXZ 00405CC0
 0003:00001DCE       ?_STD_VEDBTR_EndServiceThread@@YAXXZ 00404DCE
 0003:00000FAC       ?exitFromMain@@YAXXZ       00403FAC
 0004:00001ECC       ?exitval@@3HA              00408ECC
 0004:00001598       ?pMainHeap@RTLHeap@@0PAV1@A 00408598
 0004:00001420       ?pMainHeap@RTLMultiPool@@0PAV1@A 00408420
 0004:00001594       ?pPools@RTLPool@@0PAV1@A   00408594
 0004:00000D30       _$ClassNwQuotaD            00407D30
 0003:0000332A  Imp  _$Classjava_io_FileOutputStream (SNJRT11.DLL.$Classjava_io_FileOutputStream)
 0003:00003342  Imp  _$Classjava_io_IOException (SNJRT11.DLL.$Classjava_io_IOException)
 0003:00003324  Imp  _$Classjava_io_PrintWriter (SNJRT11.DLL.$Classjava_io_PrintWriter)
 0003:000033CC  Imp  _$Classjava_lang_NumberFormatException (SNJRT11.DLL.$Classjava_lang_NumberFormatException)
 0003:000033D8  Imp  _$Classjava_lang_Object (SNJRT11.DLL.$Classjava_lang_Object)
 0003:00003300  Imp  _$Classjava_lang_String (SNJRT11.DLL.$Classjava_lang_String)
 0003:0000336C  Imp  _$Classjava_lang_StringBuffer (SNJRT11.DLL.$Classjava_lang_StringBuffer)
 0003:000033AE  Imp  _$Classjava_lang_System (SNJRT11.DLL.$Classjava_lang_System)
 0003:000032F4  Imp  _$Classjava_net_DatagramPacket (SNJRT11.DLL.$Classjava_net_DatagramPacket)
 0003:000032E8  Imp  _$Classjava_net_DatagramSocket (SNJRT11.DLL.$Classjava_net_DatagramSocket)
 0003:00003348  Imp  _$Classjava_text_SimpleDateFormat (SNJRT11.DLL.$Classjava_text_SimpleDateFormat)
 0003:00003354  Imp  _$Classjava_util_Date (SNJRT11.DLL.$Classjava_util_Date)
 0004:000016E0       _$NwQuotaD_VERSION_1NUMBER 004086E0
 0003:00000018       _$NwQuotaD__4clinit_5__    00403018
 0003:0000004C       _$NwQuotaD__4init_5__      0040304C
 0003:000004C0       _$NwQuotaD_dumpToFile__Ljava_lang_String_2 004034C0
 0004:000016E4       _$NwQuotaD_filter          004086E4
 0004:00000085       _$NwQuotaD_filtrePositif   00407085
 0003:000005C4       _$NwQuotaD_getCurrentDateFormated__ 004035C4
 0004:000016E8       _$NwQuotaD_logFileName     004086E8
 0003:0000060C       _$NwQuotaD_main___3Ljava_lang_String_2 0040360C
 0003:00000848       _$NwQuotaD_parseArgs___3Ljava_lang_String_2 00403848
 0004:00000080       _$NwQuotaD_port            00407080
 0004:00000084       _$NwQuotaD_showOnlyAlert   00407084
 0003:00003330  Imp  _$java_io_FileOutputStream__4init_5__Ljava_lang_String_2Z (SNJRT11.DLL.$java_io_FileOutputStream__4init_5__Ljava_lang_String_2Z)
 0003:00003336  Imp  _$java_io_PrintWriter__4init_5__Ljava_io_OutputStream_2 (SNJRT11.DLL.$java_io_PrintWriter__4init_5__Ljava_io_OutputStream_2)
 0003:00003390  Imp  _$java_lang_Integer_parseInt__Ljava_lang_String_2 (SNJRT11.DLL.$java_lang_Integer_parseInt__Ljava_lang_String_2)
 0003:000032DC  Imp  _$java_lang_Object__4init_5__ (SNJRT11.DLL.$java_lang_Object__4init_5__)
 0003:000033F6  Imp  _$java_lang_Object_clone__ (SNJRT11.DLL.$java_lang_Object_clone__)
 0003:000033F0  Imp  _$java_lang_Object_equals__Ljava_lang_Object_2 (SNJRT11.DLL.$java_lang_Object_equals__Ljava_lang_Object_2)
 0003:00003420  Imp  _$java_lang_Object_finalize__ (SNJRT11.DLL.$java_lang_Object_finalize__)
 0003:000033E4  Imp  _$java_lang_Object_getClass__ (SNJRT11.DLL.$java_lang_Object_getClass__)
 0003:000033EA  Imp  _$java_lang_Object_hashCode__ (SNJRT11.DLL.$java_lang_Object_hashCode__)
 0003:00003408  Imp  _$java_lang_Object_notifyAll__ (SNJRT11.DLL.$java_lang_Object_notifyAll__)
 0003:00003402  Imp  _$java_lang_Object_notify__ (SNJRT11.DLL.$java_lang_Object_notify__)
 0003:000033FC  Imp  _$java_lang_Object_toString__ (SNJRT11.DLL.$java_lang_Object_toString__)
 0003:0000341A  Imp  _$java_lang_Object_wait__ (SNJRT11.DLL.$java_lang_Object_wait__)
 0003:0000340E  Imp  _$java_lang_Object_wait__J (SNJRT11.DLL.$java_lang_Object_wait__J)
 0003:00003414  Imp  _$java_lang_Object_wait__JI (SNJRT11.DLL.$java_lang_Object_wait__JI)
 0003:00003372  Imp  _$java_lang_StringBuffer__4init_5__ (SNJRT11.DLL.$java_lang_StringBuffer__4init_5__)
 0003:00003366  Imp  _$java_lang_StringBuffer_append__I (SNJRT11.DLL.$java_lang_StringBuffer_append__I)
 0003:0000333C  Imp  _$java_lang_StringBuffer_append__Ljava_lang_Object_2 (SNJRT11.DLL.$java_lang_StringBuffer_append__Ljava_lang_Object_2)
 0003:0000337E  Imp  _$java_lang_StringBuffer_append__Ljava_lang_String_2 (SNJRT11.DLL.$java_lang_StringBuffer_append__Ljava_lang_String_2)
 0003:00003378  Imp  _$java_lang_StringBuffer_append__Z (SNJRT11.DLL.$java_lang_StringBuffer_append__Z)
 0003:00003384  Imp  _$java_lang_StringBuffer_toString__ (SNJRT11.DLL.$java_lang_StringBuffer_toString__)
 0003:00003312  Imp  _$java_lang_String__4init_5___3BII (SNJRT11.DLL.$java_lang_String__4init_5___3BII)
 0003:00003396  Imp  _$java_lang_String_equals__Ljava_lang_Object_2 (SNJRT11.DLL.$java_lang_String_equals__Ljava_lang_Object_2)
 0003:00003318  Imp  _$java_lang_String_indexOf__Ljava_lang_String_2 (SNJRT11.DLL.$java_lang_String_indexOf__Ljava_lang_String_2)
 0003:000033BA  Imp  _$java_lang_String_startsWith__Ljava_lang_String_2 (SNJRT11.DLL.$java_lang_String_startsWith__Ljava_lang_String_2)
 0003:000033C6  Imp  _$java_lang_String_substring__I (SNJRT11.DLL.$java_lang_String_substring__I)
 0003:000033A2  Imp  _$java_lang_String_toUpperCase__ (SNJRT11.DLL.$java_lang_String_toUpperCase__)
 0003:000033A8  Imp  _$java_lang_System_out (SNJRT11.DLL.$java_lang_System_out)
 0003:000032FA  Imp  _$java_net_DatagramPacket__4init_5___3BI (SNJRT11.DLL.$java_net_DatagramPacket__4init_5___3BI)
 0003:00003306  Imp  _$java_net_DatagramPacket_getData__ (SNJRT11.DLL.$java_net_DatagramPacket_getData__)
 0003:0000330C  Imp  _$java_net_DatagramPacket_getLength__ (SNJRT11.DLL.$java_net_DatagramPacket_getLength__)
 0003:000032EE  Imp  _$java_net_DatagramSocket__4init_5__I (SNJRT11.DLL.$java_net_DatagramSocket__4init_5__I)
 0003:00003360  Imp  _$java_text_DateFormat_format__Ljava_util_Date_2 (SNJRT11.DLL.$java_text_DateFormat_format__Ljava_util_Date_2)
 0003:0000334E  Imp  _$java_text_SimpleDateFormat__4init_5__Ljava_lang_String_2 (SNJRT11.DLL.$java_text_SimpleDateFormat__4init_5__Ljava_lang_String_2)
 0003:0000335A  Imp  _$java_util_Date__4init_5__ (SNJRT11.DLL.$java_util_Date__4init_5__)
 0003:000034BC  Imp  _CloseHandle@4       (KERNEL32.DLL.CloseHandle)
 0003:00003492  Imp  _CreateSemaphoreA@16 (KERNEL32.DLL.CreateSemaphoreA)
 0003:00003498  Imp  _CreateThread@24     (KERNEL32.DLL.CreateThread)
 0003:000034C8  Imp  _DeleteCriticalSection@4 (KERNEL32.DLL.DeleteCriticalSection)
 0003:0000344A  Imp  _EnterCriticalSection@4 (KERNEL32.DLL.EnterCriticalSection)
 0003:00003504  Imp  _ExitProcess@4       (KERNEL32.DLL.ExitProcess)
 0004:00001039       _FE_DFL_ENV                00408039
 0003:00003462  Imp  _FileTimeToDosDateTime@12 (KERNEL32.DLL.FileTimeToDosDateTime)
 0003:00003456  Imp  _FindClose@4         (KERNEL32.DLL.FindClose)
 0003:0000345C  Imp  _FindFirstFileA@8    (KERNEL32.DLL.FindFirstFileA)
 0003:00003468  Imp  _FindNextFileA@8     (KERNEL32.DLL.FindNextFileA)
 0003:000034EC  Imp  _FreeEnvironmentStringsA@4 (KERNEL32.DLL.FreeEnvironmentStringsA)
 0003:00003438  Imp  _GetACP@0            (KERNEL32.DLL.GetACP)
 0003:0000342C  Imp  _GetCPInfo@8         (KERNEL32.DLL.GetCPInfo)
 0003:00003510  Imp  _GetCommandLineA@0   (KERNEL32.DLL.GetCommandLineA)
 0003:000034DA  Imp  _GetCurrentThreadId@0 (KERNEL32.DLL.GetCurrentThreadId)
 0003:000034F8  Imp  _GetEnvironmentStrings@0 (KERNEL32.DLL.GetEnvironmentStrings)
 0003:0000348C  Imp  _GetEnvironmentVariableA@12 (KERNEL32.DLL.GetEnvironmentVariableA)
 0003:0000347A  Imp  _GetLastError@0      (KERNEL32.DLL.GetLastError)
 0003:000034E0  Imp  _GetModuleFileNameA@12 (KERNEL32.DLL.GetModuleFileNameA)
 0003:0000350A  Imp  _GetModuleHandleA@4  (KERNEL32.DLL.GetModuleHandleA)
 0003:00003432  Imp  _GetOEMCP@0          (KERNEL32.DLL.GetOEMCP)
 0003:00003474  Imp  _GetProcAddress@8    (KERNEL32.DLL.GetProcAddress)
 0003:00003444  Imp  _GetStdHandle@4      (KERNEL32.DLL.GetStdHandle)
 0003:000034D4  Imp  _GetTickCount@0      (KERNEL32.DLL.GetTickCount)
 0003:000034F2  Imp  _GetVersion@0        (KERNEL32.DLL.GetVersion)
 0003:000034C2  Imp  _InitializeCriticalSection@4 (KERNEL32.DLL.InitializeCriticalSection)
 0003:00003450  Imp  _LeaveCriticalSection@4 (KERNEL32.DLL.LeaveCriticalSection)
 0003:0000346E  Imp  _LoadLibraryA@4      (KERNEL32.DLL.LoadLibraryA)
 0003:00003516  Imp  _MessageBoxA@16      (user32.DLL.MessageBoxA)
 0003:000034E6  Imp  _MultiByteToWideChar@24 (KERNEL32.DLL.MultiByteToWideChar)
 0003:000034B0  Imp  _ReleaseSemaphore@12 (KERNEL32.DLL.ReleaseSemaphore)
 0003:000034CE  Imp  _RtlUnwind@16        (KERNEL32.DLL.RtlUnwind)
 0003:000032C4  Imp  _SNJRegisterModule   (SNJRT11.DLL.SNJRegisterModule)
 0003:000032CA  Imp  _SNJRunMain          (SNJRT11.DLL.SNJRunMain)
 0003:0000349E  Imp  _SetThreadPriority@8 (KERNEL32.DLL.SetThreadPriority)
 0003:000034AA  Imp  _Sleep@4             (KERNEL32.DLL.Sleep)
 0003:000034B6  Imp  _TerminateThread@8   (KERNEL32.DLL.TerminateThread)
 0003:000034FE  Imp  _UnhandledExceptionFilter@4 (KERNEL32.DLL.UnhandledExceptionFilter)
 0003:00003480  Imp  _VirtualAlloc@16     (KERNEL32.DLL.VirtualAlloc)
 0003:00003426  Imp  _VirtualFree@12      (KERNEL32.DLL.VirtualFree)
 0003:00003486  Imp  _VirtualProtect@16   (KERNEL32.DLL.VirtualProtect)
 0003:000034A4  Imp  _WaitForSingleObject@8 (KERNEL32.DLL.WaitForSingleObject)
 0003:0000343E  Imp  _WriteConsoleA@20    (KERNEL32.DLL.WriteConsoleA)
 0003:0000189E       __FEEXCEPT                 0040489E
 0003:000018B2       __FEROUND                  004048B2
 0003:000018D4       __InitSemaphoreSys         004048D4
 0003:000019C4       __ReleaseSemaphore         004049C4
 0003:00002C34       __SET_ERRNO                00405C34
 0003:00002BA0       __SET_NT_ERRNO             00405BA0
 0003:00001940       __WaitSemaphore            00404940
 0003:000027E4       ___SD?%___heap32_multpool_cpp2346133860_ 004057E4
 0003:000027F8       ___SI?%___heap32_multpool_cpp2346133860_ 004057F8
 0004:0000102D       ___argc                    0040802D
 0004:00001031       ___argv                    00408031
 0003:0000126C       ___build_environ           0040426C
 0003:00001E48       ___callve                  00404E48
 0003:00001BC0       ___cc_array                00404BC0
 0003:00001BC6       ___cc_handles              00404BC6
 0003:00001BCC       ___cc_handles_length       00404BCC
 0004:0000265C       ___cpp_init_ptr            0040965C
 0003:00001893       ___doserrno                00404893
 0003:00001E60       ___faterr                  00404E60
 0004:00001324       ___fp_sigfunc              00408324
 0004:000012E0       ___init_environ_ptr        004082E0
 0004:00001428       ___init_mbctype_ptr        00408428
 0003:000017A0       ___initmbctype             004047A0
 0003:00002837       ___itoa                    00405837
 0004:000013A0       ___locale_codepage         004083A0
 0004:000013A4       ___locale_ident            004083A4
 0004:0000139C       ___locale_mbsize           0040839C
 0004:0000162C       ___mb_cpinfo               0040862C
 0004:000016CC       ___mb_cpinfoN              004086CC
 0004:00001534       ___mbcodepage              00408534
 0004:00001530       ___mbcpinfo                00408530
 0004:00001538       ___mblcid                  00408538
 0004:00001EC0       ___module_handle           00408EC0
 0003:00001E30       ___rtl_clean_cppexceptions 00404E30
 0004:00001330       ___rtl_criticalsection     00408330
 0003:00001E18       ___rtl_init_cppexceptions  00404E18
 0004:00001328       ___sigill_sigfunc          00408328
 0004:0000132C       ___sigsegv_sigfunc         0040832C
 0004:00000FDC       ___terminate_done          00407FDC
 0004:000012F8       ___thdtbl                  004082F8
 0003:00001842       ___threadid                00404842
 0004:00001398       ___ve_debughook            00408398
 0004:00001035       ___wargv                   00408035
 0004:00000FBC       ___wildcard                00407FBC
 0003:00000E0C       ___xcfilter                00403E0C
 0004:00001310       __acmdln                   00408310
 0004:00000FC4       __acrtused_con             00407FC4
 0003:000024C8       __addthreadtableentry      004054C8
 0003:000018BC       __allocinit                004048BC
 0004:0000102D       __argc                     0040802D
 0004:00001031       __argv                     00408031
 0004:00000FE4       __atexit_max               00407FE4
 0004:00001DB4       __atexit_tbl               00408DB4
 0004:00000FE0       __atexitp                  00407FE0
 0004:00001314       __atopsp                   00408314
 0003:00001A84       __call_except_block        00404A84
 0003:00001030       __cinit                    00404030
 0003:00001A50       __clearbss                 00404A50
 0004:0000110F       __cppeh_sv                 0040810F
 0004:00000FE8       __cpumode                  00407FE8
 0003:00001B9C       __delete_rtl_critsection   00404B9C
 0003:000010F2       __dodtors                  004040F2
 0004:000010CF       __doserrno                 004080CF
 0004:00001700       __edata                    00408700
 0004:00002670       __end                      00409670
 0004:000012D8       __environ                  004082D8
 0004:00001025       __envptr                   00408025
 0003:0000188A       __errno                    0040488A
 0003:0000187A       __errno_set                0040487A
 0003:00000D1C       __except_handler3          00403D1C
 0000:00000000  Abs  __except_list              00000000
 0003:00000E00       __exit                     00403E00
 0003:000031D4       __fatexit                  004061D4
 0004:00001EC8       __fcloseallp               00408EC8
 0004:0000108B       __fe_cur_env               0040808B
 0003:000017FD       __getthreaddata            004047FD
 0003:00001AC0       __global_unwind            00404AC0
 0004:00002434       __hdlSemHandles            00409434
 0004:00001EC4       __hookexitp                00408EC4
 0004:00001ED0       __iSemLockCtrs             00408ED0
 0004:0000220C       __iSemNestCount            0040920C
 0004:00001FE4       __iSemThreadIds            00408FE4
 0002:00000CEC       __imp__$Classjava_io_FileOutputStream 00402CEC
 0002:00000CFC       __imp__$Classjava_io_IOException 00402CFC
 0002:00000CE8       __imp__$Classjava_io_PrintWriter 00402CE8
 0002:00000D58       __imp__$Classjava_lang_NumberFormatException 00402D58
 0002:00000D60       __imp__$Classjava_lang_Object 00402D60
 0002:00000CD0       __imp__$Classjava_lang_String 00402CD0
 0002:00000D18       __imp__$Classjava_lang_StringBuffer 00402D18
 0002:00000D44       __imp__$Classjava_lang_System 00402D44
 0002:00000CC8       __imp__$Classjava_net_DatagramPacket 00402CC8
 0002:00000CC0       __imp__$Classjava_net_DatagramSocket 00402CC0
 0002:00000D00       __imp__$Classjava_text_SimpleDateFormat 00402D00
 0002:00000D08       __imp__$Classjava_util_Date 00402D08
 0002:00000D40       __imp__$java_lang_System_out 00402D40
 0002:00000DFC       __imp__CloseHandle@4       00402DFC
 0002:00000DE0       __imp__CreateSemaphoreA@16 00402DE0
 0002:00000DE4       __imp__CreateThread@24     00402DE4
 0002:00000E04       __imp__DeleteCriticalSection@4 00402E04
 0002:00000DB0       __imp__EnterCriticalSection@4 00402DB0
 0002:00000DC0       __imp__FileTimeToDosDateTime@12 00402DC0
 0002:00000DB8       __imp__FindClose@4         00402DB8
 0002:00000DBC       __imp__FindFirstFileA@8    00402DBC
 0002:00000DC4       __imp__FindNextFileA@8     00402DC4
 0002:00000DA4       __imp__GetACP@0            00402DA4
 0002:00000D9C       __imp__GetCPInfo@8         00402D9C
 0002:00000E34       __imp__GetCommandLineA@0   00402E34
 0002:00000DDC       __imp__GetEnvironmentVariableA@12 00402DDC
 0002:00000DD0       __imp__GetLastError@0      00402DD0
 0002:00000E14       __imp__GetModuleFileNameA@12 00402E14
 0002:00000E30       __imp__GetModuleHandleA@4  00402E30
 0002:00000DA0       __imp__GetOEMCP@0          00402DA0
 0002:00000DAC       __imp__GetStdHandle@4      00402DAC
 0002:00000E0C       __imp__GetTickCount@0      00402E0C
 0002:00000E00       __imp__InitializeCriticalSection@4 00402E00
 0002:00000DB4       __imp__LeaveCriticalSection@4 00402DB4
 0002:00000E3C       __imp__MessageBoxA@16      00402E3C
 0002:00000E18       __imp__MultiByteToWideChar@24 00402E18
 0002:00000DF4       __imp__ReleaseSemaphore@12 00402DF4
 0002:00000DE8       __imp__SetThreadPriority@8 00402DE8
 0002:00000DF0       __imp__Sleep@4             00402DF0
 0002:00000DF8       __imp__TerminateThread@8   00402DF8
 0002:00000E28       __imp__UnhandledExceptionFilter@4 00402E28
 0002:00000DD4       __imp__VirtualAlloc@16     00402DD4
 0002:00000D98       __imp__VirtualFree@12      00402D98
 0002:00000DEC       __imp__WaitForSingleObject@8 00402DEC
 0002:00000DA8       __imp__WriteConsoleA@20    00402DA8
 0002:00000D64       __imp___vtbl_$Classjava_lang_Class 00402D64
 0003:00001B7C       __init_rtl_critsection     00404B7C
 0003:0000247C       __ismbblead                0040547C
 0003:0000339C  Imp  __j_arraybounds@0    (SNJRT11.DLL.__j_arraybounds@0)
 0003:000033C0  Imp  __j_classinit        (SNJRT11.DLL._j_classinit)
 0003:0000331E  Imp  __j_local_unwind2    (SNJRT11.DLL._j_local_unwind2)
 0003:0000338A  Imp  __j_new@4            (SNJRT11.DLL.__j_new@4)
 0003:000032E2  Imp  __j_newarray@8       (SNJRT11.DLL.__j_newarray@8)
 0003:000033B4  Imp  __j_stringfix        (SNJRT11.DLL._j_stringfix)
 0003:000033D2  Imp  __java_framehandler  (SNJRT11.DLL._java_framehandler)
 0003:00000010       __java_main                00403010
 0004:00000FC0       __jrtused                  00407FC0
 0003:00001AA0       __local_except_handler     00404AA0
 0003:00001AE8       __local_unwind             00404AE8
 0004:0000142C       __mbctype                  0040842C
 0003:000020CC       __mbschr                   004050CC
 0003:0000286C       __opti_stosd               0040586C
 0004:00000FFA       __osmode                   00407FFA
 0004:00000FF2       __osver                    00407FF2
 0004:00000FEA       __pgmptr                   00407FEA
 0003:00001122       __semerr                   00404122
 0003:000014C0       __setargv                  004044C0
 0003:00001E68       __setenvp                  00404E68
 0003:00002A7C       __setmbcp                  00405A7C
 0004:00002660       __szSemPrefix              00409660
 0004:00000FE6       __tab_size                 00407FE6
 0003:000017F3       __thderr                   004047F3
 0004:00001043       __thread1                  00408043
 0003:000017C0       __thread_init              004047C0
 0003:00001D25       __vedbtr_CreateServiceThread 00404D25
 0004:00000F80       __vtbl_$ClassNwQuotaD      00407F80
 0003:000033DE  Imp  __vtbl_$Classjava_lang_Class (SNJRT11.DLL._vtbl_$Classjava_lang_Class)
 0004:00001035       __wargv                    00408035
 0004:000012DC       __wenviron                 004082DC
 0004:00001029       __wenvptr                  00408029
 0003:00002944       __win32_faterr             00405944
 0003:000028F8       __win32_stderrmsg          004058F8
 0004:00000FF7       __winmajor                 00407FF7
 0004:00000FF6       __winminor                 00407FF6
 0004:00000FF6       __winver                   00407FF6
 0004:00000FEE       __wpgmptr                  00407FEE
 0004:00000020       __xc_a                     00407020
 0004:00000030       __xc_z                     00407030
 0004:00000000       __xi_a                     00407000
 0004:00000010       __xi_z                     00407010
 0004:00000040       __xp_a                     00407040
 0004:00000050       __xp_z                     00407050
 0004:00000060       __xt_a                     00407060
 0004:00000070       __xt_z                     00407070
 0003:00002490       _calloc                    00405490
 0004:00001700       _edata                     00408700
 0004:00002670       _end                       00409670
 0004:00001053       _errno                     00408053
 0003:00000F04       _exit                      00403F04
 0003:000023E0       _findfirst                 004053E0
 0003:00002424       _findnext                  00405424
 0003:00002080       _free                      00405080
 0003:00002810       _itoa                      00405810
 0003:00000FBB       _main                      00403FBB
 0003:00000C50       _mainCRTStartup            00403C50
 0003:00001F94       _malloc                    00404F94
 0003:00002180       _memcpy                    00405180
 0003:00002180       _memmove                   00405180
 0003:000028A0       _memset                    004058A0
 0003:00001FEC       _realloc                   00404FEC
 0003:00003220       _sbrk                      00406220
 0003:00002440       _strcat                    00405440
 0003:00001F40       _strchr                    00404F40
 0003:00001E7C       _strcpy                    00404E7C
 0003:00002048       _strdup                    00405048
 0003:00001EE0       _strlen                    00404EE0
 0003:000032D0  Imp  _sysAtexit           (SNJRT11.DLL.sysAtexit)
 0003:000032D6  Imp  _sysExit             (SNJRT11.DLL.sysExit)

  Address         Publics by Value              Rva+Base

 0000:00000000  Abs  __except_list              00000000
 0002:00000CC0       __imp__$Classjava_net_DatagramSocket 00402CC0
 0002:00000CC8       __imp__$Classjava_net_DatagramPacket 00402CC8
 0002:00000CD0       __imp__$Classjava_lang_String 00402CD0
 0002:00000CE8       __imp__$Classjava_io_PrintWriter 00402CE8
 0002:00000CEC       __imp__$Classjava_io_FileOutputStream 00402CEC
 0002:00000CFC       __imp__$Classjava_io_IOException 00402CFC
 0002:00000D00       __imp__$Classjava_text_SimpleDateFormat 00402D00
 0002:00000D08       __imp__$Classjava_util_Date 00402D08
 0002:00000D18       __imp__$Classjava_lang_StringBuffer 00402D18
 0002:00000D40       __imp__$java_lang_System_out 00402D40
 0002:00000D44       __imp__$Classjava_lang_System 00402D44
 0002:00000D58       __imp__$Classjava_lang_NumberFormatException 00402D58
 0002:00000D60       __imp__$Classjava_lang_Object 00402D60
 0002:00000D64       __imp___vtbl_$Classjava_lang_Class 00402D64
 0002:00000D98       __imp__VirtualFree@12      00402D98
 0002:00000D9C       __imp__GetCPInfo@8         00402D9C
 0002:00000DA0       __imp__GetOEMCP@0          00402DA0
 0002:00000DA4       __imp__GetACP@0            00402DA4
 0002:00000DA8       __imp__WriteConsoleA@20    00402DA8
 0002:00000DAC       __imp__GetStdHandle@4      00402DAC
 0002:00000DB0       __imp__EnterCriticalSection@4 00402DB0
 0002:00000DB4       __imp__LeaveCriticalSection@4 00402DB4
 0002:00000DB8       __imp__FindClose@4         00402DB8
 0002:00000DBC       __imp__FindFirstFileA@8    00402DBC
 0002:00000DC0       __imp__FileTimeToDosDateTime@12 00402DC0
 0002:00000DC4       __imp__FindNextFileA@8     00402DC4
 0002:00000DD0       __imp__GetLastError@0      00402DD0
 0002:00000DD4       __imp__VirtualAlloc@16     00402DD4
 0002:00000DDC       __imp__GetEnvironmentVariableA@12 00402DDC
 0002:00000DE0       __imp__CreateSemaphoreA@16 00402DE0
 0002:00000DE4       __imp__CreateThread@24     00402DE4
 0002:00000DE8       __imp__SetThreadPriority@8 00402DE8
 0002:00000DEC       __imp__WaitForSingleObject@8 00402DEC
 0002:00000DF0       __imp__Sleep@4             00402DF0
 0002:00000DF4       __imp__ReleaseSemaphore@12 00402DF4
 0002:00000DF8       __imp__TerminateThread@8   00402DF8
 0002:00000DFC       __imp__CloseHandle@4       00402DFC
 0002:00000E00       __imp__InitializeCriticalSection@4 00402E00
 0002:00000E04       __imp__DeleteCriticalSection@4 00402E04
 0002:00000E0C       __imp__GetTickCount@0      00402E0C
 0002:00000E14       __imp__GetModuleFileNameA@12 00402E14
 0002:00000E18       __imp__MultiByteToWideChar@24 00402E18
 0002:00000E28       __imp__UnhandledExceptionFilter@4 00402E28
 0002:00000E30       __imp__GetModuleHandleA@4  00402E30
 0002:00000E34       __imp__GetCommandLineA@0   00402E34
 0002:00000E3C       __imp__MessageBoxA@16      00402E3C
 0003:00000010       __java_main                00403010
 0003:00000018       _$NwQuotaD__4clinit_5__    00403018
 0003:0000004C       _$NwQuotaD__4init_5__      0040304C
 0003:000004C0       _$NwQuotaD_dumpToFile__Ljava_lang_String_2 004034C0
 0003:000005C4       _$NwQuotaD_getCurrentDateFormated__ 004035C4
 0003:0000060C       _$NwQuotaD_main___3Ljava_lang_String_2 0040360C
 0003:00000848       _$NwQuotaD_parseArgs___3Ljava_lang_String_2 00403848
 0003:00000C50       _mainCRTStartup            00403C50
 0003:00000D1C       __except_handler3          00403D1C
 0003:00000E00       __exit                     00403E00
 0003:00000E0C       ___xcfilter                00403E0C
 0003:00000F04       _exit                      00403F04
 0003:00000FAC       ?exitFromMain@@YAXXZ       00403FAC
 0003:00000FBB       _main                      00403FBB
 0003:00001030       __cinit                    00404030
 0003:000010F2       __dodtors                  004040F2
 0003:00001122       __semerr                   00404122
 0003:0000126C       ___build_environ           0040426C
 0003:000014C0       __setargv                  004044C0
 0003:000017A0       ___initmbctype             004047A0
 0003:000017C0       __thread_init              004047C0
 0003:000017F3       __thderr                   004047F3
 0003:000017FD       __getthreaddata            004047FD
 0003:00001842       ___threadid                00404842
 0003:0000187A       __errno_set                0040487A
 0003:0000188A       __errno                    0040488A
 0003:00001893       ___doserrno                00404893
 0003:0000189E       __FEEXCEPT                 0040489E
 0003:000018B2       __FEROUND                  004048B2
 0003:000018BC       __allocinit                004048BC
 0003:000018D4       __InitSemaphoreSys         004048D4
 0003:00001940       __WaitSemaphore            00404940
 0003:000019C4       __ReleaseSemaphore         004049C4
 0003:00001A50       __clearbss                 00404A50
 0003:00001A84       __call_except_block        00404A84
 0003:00001AA0       __local_except_handler     00404AA0
 0003:00001AC0       __global_unwind            00404AC0
 0003:00001AE8       __local_unwind             00404AE8
 0003:00001B7C       __init_rtl_critsection     00404B7C
 0003:00001B9C       __delete_rtl_critsection   00404B9C
 0003:00001BC0       ___cc_array                00404BC0
 0003:00001BC6       ___cc_handles              00404BC6
 0003:00001BCC       ___cc_handles_length       00404BCC
 0003:00001D25       __vedbtr_CreateServiceThread 00404D25
 0003:00001DCE       ?_STD_VEDBTR_EndServiceThread@@YAXXZ 00404DCE
 0003:00001E18       ___rtl_init_cppexceptions  00404E18
 0003:00001E30       ___rtl_clean_cppexceptions 00404E30
 0003:00001E48       ___callve                  00404E48
 0003:00001E60       ___faterr                  00404E60
 0003:00001E68       __setenvp                  00404E68
 0003:00001E7C       _strcpy                    00404E7C
 0003:00001EE0       _strlen                    00404EE0
 0003:00001F40       _strchr                    00404F40
 0003:00001F94       _malloc                    00404F94
 0003:00001FEC       _realloc                   00404FEC
 0003:00002048       _strdup                    00405048
 0003:00002080       _free                      00405080
 0003:000020CC       __mbschr                   004050CC
 0003:00002180       _memmove                   00405180
 0003:00002180       _memcpy                    00405180
 0003:000023E0       _findfirst                 004053E0
 0003:00002424       _findnext                  00405424
 0003:00002440       _strcat                    00405440
 0003:0000247C       __ismbblead                0040547C
 0003:00002490       _calloc                    00405490
 0003:000024C8       __addthreadtableentry      004054C8
 0003:00002568       ??0RTLMultiPool@@QAE@II@Z  00405568
 0003:000025EC       ??1RTLMultiPool@@QAE@XZ    004055EC
 0003:000025F0       ?Alloc@RTLMultiPool@@QAEPAXK@Z 004055F0
 0003:00002640       ?Realloc@RTLMultiPool@@QAEPAXPAXK@Z 00405640
 0003:00002760       ?SelectFree@RTLMultiPool@@AAEXPAX@Z 00405760
 0003:0000279C       ?Free@RTLMultiPool@@QAEXPAX@Z 0040579C
 0003:000027B4       ?CreateMainHeap@RTLMultiPool@@SAXXZ 004057B4
 0003:000027E4       ___SD?%___heap32_multpool_cpp2346133860_ 004057E4
 0003:000027F8       ___SI?%___heap32_multpool_cpp2346133860_ 004057F8
 0003:00002810       _itoa                      00405810
 0003:00002837       ___itoa                    00405837
 0003:0000286C       __opti_stosd               0040586C
 0003:000028A0       _memset                    004058A0
 0003:000028F8       __win32_stderrmsg          004058F8
 0003:00002944       __win32_faterr             00405944
 0003:00002A7C       __setmbcp                  00405A7C
 0003:00002BA0       __SET_NT_ERRNO             00405BA0
 0003:00002C34       __SET_ERRNO                00405C34
 0003:00002C5C       ??0RTLPool@@QAE@II@Z       00405C5C
 0003:00002CC0       ?ThreadNewBlock@RTLPool@@AAEXXZ 00405CC0
 0003:00002D4C       ?Alloc@RTLPool@@QAEPAXXZ   00405D4C
 0003:00002D7C       ?Free@RTLPool@@QAEXPAX@Z   00405D7C
 0003:00002D90       ??0RTLHeap@@QAE@XZ         00405D90
 0003:00002DAC       ?FixSize@RTLHeap@@AAEII@Z  00405DAC
 0003:00002DE8       ?Alloc@RTLHeap@@QAEPAXK@Z  00405DE8
 0003:00002E4C       ?Realloc@RTLHeap@@QAEPAXPAXK@Z 00405E4C
 0003:00002F20       ?MoreCore@RTLHeap@@AAEPAVRTLHeapBlock@@I@Z 00405F20
 0003:00002F90       ?Free@RTLHeap@@QAEXPAX@Z   00405F90
 0003:00002FE0       ??0RTLHeapBlockHeader@@QAE@I@Z 00405FE0
 0003:00002FFC       ??0RTLHeapBlock@@QAE@XZ    00405FFC
 0003:00003010       ??0RTLHeapBlock@@QAE@IAAV0@@Z 00406010
 0003:00003030       ?InsertAfter@RTLHeapBlock@@QAEXAAV1@@Z 00406030
 0003:00003058       ?MergeBackward@RTLHeapBlock@@QAEHXZ 00406058
 0003:00003098       ?MergeForward@RTLHeapBlock@@QAEHXZ 00406098
 0003:000030E4       ?GetNext@RTLHeapBlock@@QAEAAV1@XZ 004060E4
 0003:000030EC       ?Remove@RTLHeapBlock@@QAEXXZ 004060EC
 0003:00003108       ?Claim@RTLHeapBlock@@QAEHI@Z 00406108
 0003:0000313C       ?Reclaim@RTLHeapBlock@@QAEHIAAV1@@Z 0040613C
 0003:000031B0       ?CreateMainHeap@RTLHeap@@SAXXZ 004061B0
 0003:000031D4       __fatexit                  004061D4
 0003:00003220       _sbrk                      00406220
 0003:000032C4  Imp  _SNJRegisterModule   (SNJRT11.DLL.SNJRegisterModule)
 0003:000032CA  Imp  _SNJRunMain          (SNJRT11.DLL.SNJRunMain)
 0003:000032D0  Imp  _sysAtexit           (SNJRT11.DLL.sysAtexit)
 0003:000032D6  Imp  _sysExit             (SNJRT11.DLL.sysExit)
 0003:000032DC  Imp  _$java_lang_Object__4init_5__ (SNJRT11.DLL.$java_lang_Object__4init_5__)
 0003:000032E2  Imp  __j_newarray@8       (SNJRT11.DLL.__j_newarray@8)
 0003:000032E8  Imp  _$Classjava_net_DatagramSocket (SNJRT11.DLL.$Classjava_net_DatagramSocket)
 0003:000032EE  Imp  _$java_net_DatagramSocket__4init_5__I (SNJRT11.DLL.$java_net_DatagramSocket__4init_5__I)
 0003:000032F4  Imp  _$Classjava_net_DatagramPacket (SNJRT11.DLL.$Classjava_net_DatagramPacket)
 0003:000032FA  Imp  _$java_net_DatagramPacket__4init_5___3BI (SNJRT11.DLL.$java_net_DatagramPacket__4init_5___3BI)
 0003:00003300  Imp  _$Classjava_lang_String (SNJRT11.DLL.$Classjava_lang_String)
 0003:00003306  Imp  _$java_net_DatagramPacket_getData__ (SNJRT11.DLL.$java_net_DatagramPacket_getData__)
 0003:0000330C  Imp  _$java_net_DatagramPacket_getLength__ (SNJRT11.DLL.$java_net_DatagramPacket_getLength__)
 0003:00003312  Imp  _$java_lang_String__4init_5___3BII (SNJRT11.DLL.$java_lang_String__4init_5___3BII)
 0003:00003318  Imp  _$java_lang_String_indexOf__Ljava_lang_String_2 (SNJRT11.DLL.$java_lang_String_indexOf__Ljava_lang_String_2)
 0003:0000331E  Imp  __j_local_unwind2    (SNJRT11.DLL._j_local_unwind2)
 0003:00003324  Imp  _$Classjava_io_PrintWriter (SNJRT11.DLL.$Classjava_io_PrintWriter)
 0003:0000332A  Imp  _$Classjava_io_FileOutputStream (SNJRT11.DLL.$Classjava_io_FileOutputStream)
 0003:00003330  Imp  _$java_io_FileOutputStream__4init_5__Ljava_lang_String_2Z (SNJRT11.DLL.$java_io_FileOutputStream__4init_5__Ljava_lang_String_2Z)
 0003:00003336  Imp  _$java_io_PrintWriter__4init_5__Ljava_io_OutputStream_2 (SNJRT11.DLL.$java_io_PrintWriter__4init_5__Ljava_io_OutputStream_2)
 0003:0000333C  Imp  _$java_lang_StringBuffer_append__Ljava_lang_Object_2 (SNJRT11.DLL.$java_lang_StringBuffer_append__Ljava_lang_Object_2)
 0003:00003342  Imp  _$Classjava_io_IOException (SNJRT11.DLL.$Classjava_io_IOException)
 0003:00003348  Imp  _$Classjava_text_SimpleDateFormat (SNJRT11.DLL.$Classjava_text_SimpleDateFormat)
 0003:0000334E  Imp  _$java_text_SimpleDateFormat__4init_5__Ljava_lang_String_2 (SNJRT11.DLL.$java_text_SimpleDateFormat__4init_5__Ljava_lang_String_2)
 0003:00003354  Imp  _$Classjava_util_Date (SNJRT11.DLL.$Classjava_util_Date)
 0003:0000335A  Imp  _$java_util_Date__4init_5__ (SNJRT11.DLL.$java_util_Date__4init_5__)
 0003:00003360  Imp  _$java_text_DateFormat_format__Ljava_util_Date_2 (SNJRT11.DLL.$java_text_DateFormat_format__Ljava_util_Date_2)
 0003:00003366  Imp  _$java_lang_StringBuffer_append__I (SNJRT11.DLL.$java_lang_StringBuffer_append__I)
 0003:0000336C  Imp  _$Classjava_lang_StringBuffer (SNJRT11.DLL.$Classjava_lang_StringBuffer)
 0003:00003372  Imp  _$java_lang_StringBuffer__4init_5__ (SNJRT11.DLL.$java_lang_StringBuffer__4init_5__)
 0003:00003378  Imp  _$java_lang_StringBuffer_append__Z (SNJRT11.DLL.$java_lang_StringBuffer_append__Z)
 0003:0000337E  Imp  _$java_lang_StringBuffer_append__Ljava_lang_String_2 (SNJRT11.DLL.$java_lang_StringBuffer_append__Ljava_lang_String_2)
 0003:00003384  Imp  _$java_lang_StringBuffer_toString__ (SNJRT11.DLL.$java_lang_StringBuffer_toString__)
 0003:0000338A  Imp  __j_new@4            (SNJRT11.DLL.__j_new@4)
 0003:00003390  Imp  _$java_lang_Integer_parseInt__Ljava_lang_String_2 (SNJRT11.DLL.$java_lang_Integer_parseInt__Ljava_lang_String_2)
 0003:00003396  Imp  _$java_lang_String_equals__Ljava_lang_Object_2 (SNJRT11.DLL.$java_lang_String_equals__Ljava_lang_Object_2)
 0003:0000339C  Imp  __j_arraybounds@0    (SNJRT11.DLL.__j_arraybounds@0)
 0003:000033A2  Imp  _$java_lang_String_toUpperCase__ (SNJRT11.DLL.$java_lang_String_toUpperCase__)
 0003:000033A8  Imp  _$java_lang_System_out (SNJRT11.DLL.$java_lang_System_out)
 0003:000033AE  Imp  _$Classjava_lang_System (SNJRT11.DLL.$Classjava_lang_System)
 0003:000033B4  Imp  __j_stringfix        (SNJRT11.DLL._j_stringfix)
 0003:000033BA  Imp  _$java_lang_String_startsWith__Ljava_lang_String_2 (SNJRT11.DLL.$java_lang_String_startsWith__Ljava_lang_String_2)
 0003:000033C0  Imp  __j_classinit        (SNJRT11.DLL._j_classinit)
 0003:000033C6  Imp  _$java_lang_String_substring__I (SNJRT11.DLL.$java_lang_String_substring__I)
 0003:000033CC  Imp  _$Classjava_lang_NumberFormatException (SNJRT11.DLL.$Classjava_lang_NumberFormatException)
 0003:000033D2  Imp  __java_framehandler  (SNJRT11.DLL._java_framehandler)
 0003:000033D8  Imp  _$Classjava_lang_Object (SNJRT11.DLL.$Classjava_lang_Object)
 0003:000033DE  Imp  __vtbl_$Classjava_lang_Class (SNJRT11.DLL._vtbl_$Classjava_lang_Class)
 0003:000033E4  Imp  _$java_lang_Object_getClass__ (SNJRT11.DLL.$java_lang_Object_getClass__)
 0003:000033EA  Imp  _$java_lang_Object_hashCode__ (SNJRT11.DLL.$java_lang_Object_hashCode__)
 0003:000033F0  Imp  _$java_lang_Object_equals__Ljava_lang_Object_2 (SNJRT11.DLL.$java_lang_Object_equals__Ljava_lang_Object_2)
 0003:000033F6  Imp  _$java_lang_Object_clone__ (SNJRT11.DLL.$java_lang_Object_clone__)
 0003:000033FC  Imp  _$java_lang_Object_toString__ (SNJRT11.DLL.$java_lang_Object_toString__)
 0003:00003402  Imp  _$java_lang_Object_notify__ (SNJRT11.DLL.$java_lang_Object_notify__)
 0003:00003408  Imp  _$java_lang_Object_notifyAll__ (SNJRT11.DLL.$java_lang_Object_notifyAll__)
 0003:0000340E  Imp  _$java_lang_Object_wait__J (SNJRT11.DLL.$java_lang_Object_wait__J)
 0003:00003414  Imp  _$java_lang_Object_wait__JI (SNJRT11.DLL.$java_lang_Object_wait__JI)
 0003:0000341A  Imp  _$java_lang_Object_wait__ (SNJRT11.DLL.$java_lang_Object_wait__)
 0003:00003420  Imp  _$java_lang_Object_finalize__ (SNJRT11.DLL.$java_lang_Object_finalize__)
 0003:00003426  Imp  _VirtualFree@12      (KERNEL32.DLL.VirtualFree)
 0003:0000342C  Imp  _GetCPInfo@8         (KERNEL32.DLL.GetCPInfo)
 0003:00003432  Imp  _GetOEMCP@0          (KERNEL32.DLL.GetOEMCP)
 0003:00003438  Imp  _GetACP@0            (KERNEL32.DLL.GetACP)
 0003:0000343E  Imp  _WriteConsoleA@20    (KERNEL32.DLL.WriteConsoleA)
 0003:00003444  Imp  _GetStdHandle@4      (KERNEL32.DLL.GetStdHandle)
 0003:0000344A  Imp  _EnterCriticalSection@4 (KERNEL32.DLL.EnterCriticalSection)
 0003:00003450  Imp  _LeaveCriticalSection@4 (KERNEL32.DLL.LeaveCriticalSection)
 0003:00003456  Imp  _FindClose@4         (KERNEL32.DLL.FindClose)
 0003:0000345C  Imp  _FindFirstFileA@8    (KERNEL32.DLL.FindFirstFileA)
 0003:00003462  Imp  _FileTimeToDosDateTime@12 (KERNEL32.DLL.FileTimeToDosDateTime)
 0003:00003468  Imp  _FindNextFileA@8     (KERNEL32.DLL.FindNextFileA)
 0003:0000346E  Imp  _LoadLibraryA@4      (KERNEL32.DLL.LoadLibraryA)
 0003:00003474  Imp  _GetProcAddress@8    (KERNEL32.DLL.GetProcAddress)
 0003:0000347A  Imp  _GetLastError@0      (KERNEL32.DLL.GetLastError)
 0003:00003480  Imp  _VirtualAlloc@16     (KERNEL32.DLL.VirtualAlloc)
 0003:00003486  Imp  _VirtualProtect@16   (KERNEL32.DLL.VirtualProtect)
 0003:0000348C  Imp  _GetEnvironmentVariableA@12 (KERNEL32.DLL.GetEnvironmentVariableA)
 0003:00003492  Imp  _CreateSemaphoreA@16 (KERNEL32.DLL.CreateSemaphoreA)
 0003:00003498  Imp  _CreateThread@24     (KERNEL32.DLL.CreateThread)
 0003:0000349E  Imp  _SetThreadPriority@8 (KERNEL32.DLL.SetThreadPriority)
 0003:000034A4  Imp  _WaitForSingleObject@8 (KERNEL32.DLL.WaitForSingleObject)
 0003:000034AA  Imp  _Sleep@4             (KERNEL32.DLL.Sleep)
 0003:000034B0  Imp  _ReleaseSemaphore@12 (KERNEL32.DLL.ReleaseSemaphore)
 0003:000034B6  Imp  _TerminateThread@8   (KERNEL32.DLL.TerminateThread)
 0003:000034BC  Imp  _CloseHandle@4       (KERNEL32.DLL.CloseHandle)
 0003:000034C2  Imp  _InitializeCriticalSection@4 (KERNEL32.DLL.InitializeCriticalSection)
 0003:000034C8  Imp  _DeleteCriticalSection@4 (KERNEL32.DLL.DeleteCriticalSection)
 0003:000034CE  Imp  _RtlUnwind@16        (KERNEL32.DLL.RtlUnwind)
 0003:000034D4  Imp  _GetTickCount@0      (KERNEL32.DLL.GetTickCount)
 0003:000034DA  Imp  _GetCurrentThreadId@0 (KERNEL32.DLL.GetCurrentThreadId)
 0003:000034E0  Imp  _GetModuleFileNameA@12 (KERNEL32.DLL.GetModuleFileNameA)
 0003:000034E6  Imp  _MultiByteToWideChar@24 (KERNEL32.DLL.MultiByteToWideChar)
 0003:000034EC  Imp  _FreeEnvironmentStringsA@4 (KERNEL32.DLL.FreeEnvironmentStringsA)
 0003:000034F2  Imp  _GetVersion@0        (KERNEL32.DLL.GetVersion)
 0003:000034F8  Imp  _GetEnvironmentStrings@0 (KERNEL32.DLL.GetEnvironmentStrings)
 0003:000034FE  Imp  _UnhandledExceptionFilter@4 (KERNEL32.DLL.UnhandledExceptionFilter)
 0003:00003504  Imp  _ExitProcess@4       (KERNEL32.DLL.ExitProcess)
 0003:0000350A  Imp  _GetModuleHandleA@4  (KERNEL32.DLL.GetModuleHandleA)
 0003:00003510  Imp  _GetCommandLineA@0   (KERNEL32.DLL.GetCommandLineA)
 0003:00003516  Imp  _MessageBoxA@16      (user32.DLL.MessageBoxA)
 0004:00000000       __xi_a                     00407000
 0004:00000010       __xi_z                     00407010
 0004:00000020       __xc_a                     00407020
 0004:00000030       __xc_z                     00407030
 0004:00000040       __xp_a                     00407040
 0004:00000050       __xp_z                     00407050
 0004:00000060       __xt_a                     00407060
 0004:00000070       __xt_z                     00407070
 0004:00000080       _$NwQuotaD_port            00407080
 0004:00000084       _$NwQuotaD_showOnlyAlert   00407084
 0004:00000085       _$NwQuotaD_filtrePositif   00407085
 0004:00000D30       _$ClassNwQuotaD            00407D30
 0004:00000F80       __vtbl_$ClassNwQuotaD      00407F80
 0004:00000FBC       ___wildcard                00407FBC
 0004:00000FC0       __jrtused                  00407FC0
 0004:00000FC4       __acrtused_con             00407FC4
 0004:00000FDC       ___terminate_done          00407FDC
 0004:00000FE0       __atexitp                  00407FE0
 0004:00000FE4       __atexit_max               00407FE4
 0004:00000FE6       __tab_size                 00407FE6
 0004:00000FE8       __cpumode                  00407FE8
 0004:00000FEA       __pgmptr                   00407FEA
 0004:00000FEE       __wpgmptr                  00407FEE
 0004:00000FF2       __osver                    00407FF2
 0004:00000FF6       __winminor                 00407FF6
 0004:00000FF6       __winver                   00407FF6
 0004:00000FF7       __winmajor                 00407FF7
 0004:00000FFA       __osmode                   00407FFA
 0004:00001025       __envptr                   00408025
 0004:00001029       __wenvptr                  00408029
 0004:0000102D       __argc                     0040802D
 0004:0000102D       ___argc                    0040802D
 0004:00001031       __argv                     00408031
 0004:00001031       ___argv                    00408031
 0004:00001035       __wargv                    00408035
 0004:00001035       ___wargv                   00408035
 0004:00001039       _FE_DFL_ENV                00408039
 0004:00001043       __thread1                  00408043
 0004:00001053       _errno                     00408053
 0004:0000108B       __fe_cur_env               0040808B
 0004:000010CF       __doserrno                 004080CF
 0004:0000110F       __cppeh_sv                 0040810F
 0004:000012D8       __environ                  004082D8
 0004:000012DC       __wenviron                 004082DC
 0004:000012E0       ___init_environ_ptr        004082E0
 0004:000012F8       ___thdtbl                  004082F8
 0004:00001310       __acmdln                   00408310
 0004:00001314       __atopsp                   00408314
 0004:00001324       ___fp_sigfunc              00408324
 0004:00001328       ___sigill_sigfunc          00408328
 0004:0000132C       ___sigsegv_sigfunc         0040832C
 0004:00001330       ___rtl_criticalsection     00408330
 0004:00001398       ___ve_debughook            00408398
 0004:0000139C       ___locale_mbsize           0040839C
 0004:000013A0       ___locale_codepage         004083A0
 0004:000013A4       ___locale_ident            004083A4
 0004:00001420       ?pMainHeap@RTLMultiPool@@0PAV1@A 00408420
 0004:00001428       ___init_mbctype_ptr        00408428
 0004:0000142C       __mbctype                  0040842C
 0004:00001530       ___mbcpinfo                00408530
 0004:00001534       ___mbcodepage              00408534
 0004:00001538       ___mblcid                  00408538
 0004:00001594       ?pPools@RTLPool@@0PAV1@A   00408594
 0004:00001598       ?pMainHeap@RTLHeap@@0PAV1@A 00408598
 0004:0000162C       ___mb_cpinfo               0040862C
 0004:000016CC       ___mb_cpinfoN              004086CC
 0004:000016E0       _$NwQuotaD_VERSION_1NUMBER 004086E0
 0004:000016E4       _$NwQuotaD_filter          004086E4
 0004:000016E8       _$NwQuotaD_logFileName     004086E8
 0004:00001700       __edata                    00408700
 0004:00001700       _edata                     00408700
 0004:00001DB4       __atexit_tbl               00408DB4
 0004:00001EC0       ___module_handle           00408EC0
 0004:00001EC4       __hookexitp                00408EC4
 0004:00001EC8       __fcloseallp               00408EC8
 0004:00001ECC       ?exitval@@3HA              00408ECC
 0004:00001ED0       __iSemLockCtrs             00408ED0
 0004:00001FE4       __iSemThreadIds            00408FE4
 0004:0000220C       __iSemNestCount            0040920C
 0004:00002434       __hdlSemHandles            00409434
 0004:0000265C       ___cpp_init_ptr            0040965C
 0004:00002660       __szSemPrefix              00409660
 0004:00002670       __end                      00409670
 0004:00002670       _end                       00409670

Line numbers for H:\dev\NwQuota\daemon\NwQuotaD.obj(NwQuotaD.java) segment _TEXT

     6 0003:00400018    86 0003:0040004C    87 0003:0040007E    88 0003:00400083
    89 0003:00400092    93 0003:004000A0    95 0003:004000CC    97 0003:0040011E
   103 0003:0040014E   104 0003:0040016E   105 0003:0040017A   106 0003:004001A6
   110 0003:004001B0   113 0003:004001F2   114 0003:0040024F   115 0003:00400266
   116 0003:0040028F   117 0003:004002B5   119 0003:004002F9   121 0003:0040032A
   122 0003:00400353   123 0003:00400379   125 0003:004003BA   129 0003:004003E3
   130 0003:00400431   131 0003:0040043C   132 0003:0040047A   141 0003:004004C0
   143 0003:004004F4   144 0003:0040052C   145 0003:0040053E   146 0003:00400546
   148 0003:00400557   150 0003:004005A9   136 0003:004005C4   137 0003:004005D3
   138 0003:004005F1   139 0003:00400609    16 0003:0040060C    17 0003:00400616
    18 0003:0040063E    19 0003:0040066A    20 0003:00400672    21 0003:00400698
    22 0003:004006ED    23 0003:00400745    24 0003:0040079D    25 0003:00400833
    26 0003:00400842    28 0003:00400848    29 0003:0040086D    30 0003:00400871
    31 0003:00400883    32 0003:00400896    34 0003:004008A3    36 0003:004008CC
    38 0003:004008EC    40 0003:004008FB    42 0003:00400931    47 0003:00400935
    48 0003:00400941    49 0003:0040099D    50 0003:004009A3    51 0003:004009FF
    52 0003:00400A05    56 0003:00400A09    57 0003:00400A1F    60 0003:00400A51
    61 0003:00400A5B    62 0003:00400A87    63 0003:00400AAA    64 0003:00400ACD
    65 0003:00400AF0    66 0003:00400B13    68 0003:00400B38    69 0003:00400B4B
    70 0003:00400B5E    74 0003:00400B71    75 0003:00400B96    76 0003:00400BA7
    79 0003:00400BD3    80 0003:00400BF9    81 0003:00400C0A    83 0003:00400C36

Program entry point at 00003C50 
